:100000000C942A000C9445000C9445000C94450077
:100010000C9445000C9445000C9445000C9445004C
:100020000C9445000C9445000C9445000C9445003C
:100030000C9445000C9445000C9445000C9445002C
:100040000C9445000C9445000C9445000C9445001C
:100050000C94450011241FBECFE5D4E0DEBFCDBF18
:1000600010E0A0E6B0E0E4EFF5E002C005900D92EC
:10007000A43DB107D9F711E0A4EDB0E001C01D9295
:10008000A432B107E1F70C942C020C940000CF933A
:10009000DF93CDB7DEB781E0809338001092350052
:1000A0001092320081E08093370010923400109259
:1000B0003100DF91CF910895CF93DF93CDB7DEB7B5
:1000C00026970FB6F894DEBF0FBECDBF69837A8343
:1000D0008B839C8389819A81AB81BC819C01AD011A
:1000E000689413F8220F331F441F551F1694D1F73D
:1000F00080E092E1AAE7B0E0BC01CD010E94D80205
:10010000DA01C90101979E838D838D819927892FFB
:10011000990F990B809340008D81809329008091E5
:100120002A00886180932A0080914000866880932D
:10013000400097EF809140008923809340002696ED
:100140000FB6F894DEBF0FBECDBFDF91CF910895FB
:10015000CF93DF93CDB7DEB722970FB6F894DEBF0B
:100160000FBECDBF80912B00882334F480912C00EA
:1001700099279A83898302C01A82198289819A8178
:1001800022960FB6F894DEBF0FBECDBFDF91CF91A0
:100190000895CF93DF93CDB7DEB721970FB6F894CC
:1001A000DEBF0FBECDBF898380912B00992780725F
:1001B0009070009709F4F8CF898180932C002196E4
:1001C0000FB6F894DEBF0FBECDBFDF91CF9108957B
:1001D000CF93DF93CDB7DEB723970FB6F894DEBF8A
:1001E0000FBECDBF89838981282F33273B832A8384
:1001F0008A819B8182309105B1F02A813B81233035
:10020000310534F48A819B818130910539F024C015
:100210002A813B812330310561F01EC08091380076
:100220001092380019C080913800816080933800A6
:1002300013C080913600992781709070009739F033
:100240008EEF9091380089238093380005C080910B
:10025000380081608093380023960FB6F894DEBF93
:100260000FBECDBFDF91CF910895CF93DF93CDB770
:10027000DEB723970FB6F894DEBF0FBECDBF9A83CB
:1002800089831B828B81282F332789819A81F901E9
:10029000E80FF91F8081882321F08B818F5F8B838A
:1002A000F1CF8B81992723960FB6F894DEBF0FBE4E
:1002B000CDBFDF91CF910895CF93DF93CDB7DEB758
:1002C00025970FB6F894DEBF0FBECDBF9A83898302
:1002D00089819A810E9435018B831C829C818B814C
:1002E000981788F48C81282F332789819A81F90106
:1002F000E80FF91F80818D838D810E94C9008C8158
:100300008F5F8C83EBCF60E670E089819A810E94D9
:10031000D10225960FB6F894DEBF0FBECDBFDF9198
:10032000CF910895CF93DF93CDB7DEB725970FB662
:10033000F894DEBF0FBECDBF9A83898389819A81ED
:100340000E9435018B831C829C818B81981788F4D5
:100350008C81282F332789819A81F901E80FF91FB1
:1003600080818D838D810E94C9008C818F5F8C83F9
:10037000EBCF60E670E089819A810E94D1028AE029
:100380000E94C9008DE00E94C90025960FB6F8941E
:10039000DEBF0FBECDBFDF91CF910895CF93DF9326
:1003A000CDB7DEB726970FB6F894DEBF0FBECDBF30
:1003B0001C82809136008B8380E690E00E9492013F
:1003C00061E670E084ED90E00E94D10284ED90E05F
:1003D0000E9492018C81882399F50E94A8008C8349
:1003E0001E821D828C81882321F421E030E03E832F
:1003F0002D838091360099279C01329522952F708C
:1004000023273F70232781E090E082279327817084
:1004100090702D813E81822393230097D9F283E04F
:100420000E94E80080E29EE49A83898389819A8110
:10043000009781F289819A8101979A838983F6CF07
:100440008B818093380026960FB6F894DEBF0FBEDE
:10045000CDBFDF91CF910895CBE5D4E0DEBFCDBF16
:100460000E94470060E875E280E090E00E945C0036
:100470001982198281E08A8380E690E00E949201CD
:100480006FE670E084ED90E00E94D10284ED90E090
:100490000E94920164E770E084ED90E00E94D10236
:1004A00084ED90E00E9492016EE770E084ED90E0B0
:1004B0000E94D10284ED90E00E94920169E870E010
:1004C00084ED90E00E94D10284ED90E00E949201C0
:1004D00067E970E084ED90E00E94D10284ED90E045
:1004E0000E94920163EB70E084ED90E00E94D102E3
:1004F00084ED90E00E945C018A81882309F4B9CFE1
:100500000E94A80089838981882319F089818053FA
:1005100089838981882381F31A828981282F33274F
:100520003C832B838B819C8182309105F1F02B8160
:100530003C812330310534F48B819C8181309105DD
:1005400061F02AC02B813C8123303105B1F08B81D1
:100550009C8184309105C9F01FC089810E94E80008
:1005600080E690E00E949201C7CF89810E94E80056
:1005700080E690E00E949201BFCF89810E94E8004E
:1005800080E690E00E949201B7CF0E94CE0180E603
:1005900090E00E949201B0CF83EC90E00E94920123
:1005A000ABCFFB01DC0101900D920020E1F7089533
:1005B000A1E21A2EAA1BBB1BFD010DC0AA1FBB1F67
:1005C000EE1FFF1FA217B307E407F50720F0A21BD9
:1005D000B30BE40BF50B661F771F881F991F1A9446
:1005E00069F760957095809590959B01AC01BD0170
:0405F000CF0108959A
:1005F40000507265737320616E79204B6579004DEC
:10060400656E75003129204C6564204F4E003229F7
:10061400204C6564204F464600332920546F676799
:100624006C65204C656400342920486F6C6420425A
:100634007574746F6E20746F20426C696E6B204CFD
:1006440065640043686F6F736520416374696F6EFE
:100654003A20004E6F207375636820616374696F7C
:040664006E2E0000F6
:00000001FF
